:1000000051C100006DC100006BC1000069C100005A
:1000100067C1000065C1000063C1000061C100004C
:100020005FC100005DC10000D5C6000059C10000DD
:1000300057C1000055C1000053C1000051C100006C
:100040004FC100004DC100004BC1000049C100007C
:1000500047C100008BC2000043C1000041C1000045
:100060003FC100003DC100003BC1000039C100009C
:1000700037C1000035C1000033C1000031C10000AC
:100080002FC100002DC100002BC1000029C10000BC
:1000900027C1000025C100004D6963726F70686F51
:1000A0006E6520456E756D6572617465642E0D0A0E
:1000B000001B5B33316D436F756C64206E6F742071
:1000C00073657420616C7465726E61746976652005
:1000D00073747265616D696E6720696E74657266AE
:1000E0006163652073657474696E672E0D0A202D37
:1000F0002D204572726F7220436F64653A2025642B
:100100000D0A1B5B33376D001B5B33316D436F6E24
:1001100074726F6C204572726F7220285365742060
:10012000436F6E66696775726174696F6E292E0D13
:100130000A202D2D204572726F7220436F64653A3C
:100140002025640D0A1B5B33376D00202D2D2045C3
:1001500072726F7220436F64653A2025640D0A1B2A
:100160005B33376D001B5B33316D496E76616C69B3
:1001700064204465766963652E0D0A001B5B33318C
:100180006D436F6E74726F6C204572726F722028AF
:1001900047657420436F6E66696775726174696F35
:1001A0006E292E0D0A0047657474696E6720436FCF
:1001B0006E66696720446174612E0D0A001B5B3313
:1001C000316D44657620456E756D204572726F7293
:1001D0000D0A202D2D204572726F7220436F6465C9
:1001E0002025640D0A202D2D205375622045727242
:1001F0006F7220436F64652025640D0A202D2D2029
:10020000496E2053746174652025640D0A1B5B33AD
:10021000376D001B5B33316D486F7374204D6F6415
:1002200065204572726F720D0A202D2D2045727265
:100230006F7220436F64652025640D0A1B5B3337A2
:100240006D001B5B33326D44657669636520556EC6
:1002500061747461636865642E0D0A1B5B33376DCE
:10026000001B5B33326D44657669636520417474AD
:1002700061636865642E0D0A1B5B33376D001B5B81
:1002800033366D417564696F20486F73742044651F
:100290006D6F2072756E6E696E672E0D0A1B5B3373
:1002A000376D000011241FBECFEFD0E2DEBFCDBFFF
:1002B00011E0A0E0B1E0EAEFF8E100E00BBF02C01E
:1002C00007900D92AC31B107D9F711E0ACE1B1E084
:1002D00001C01D92A034B107E1F73ED10C947B0C14
:1002E0008FCE9BB19F70982B9BB9089584B7877F61
:1002F00084BF28E10FB6F89420936000109260004C
:100300000FBE90E080E80FB6F89480936100909360
:1003100061000FBE83E390E09093CD008093CC000A
:1003200086E08093CA001092C8002093C900539AB7
:100330005A9A8AB1806F8AB98BB18F708BB934D5D4
:10034000ECE2F1E0F0933B01E0933A01F0933D01E0
:10035000E0933C018EE0DF011D928A95E9F783E08E
:1003600080932F0185E699E09093350180933401C5
:100370008EE699E09093370180933601089581E6E7
:1003800092E0DED780EAADCF82E492E0D9D780E177
:10039000A8CF80E6A6CFDF93CF930F92CDB7DEB77D
:1003A00089839CD400D000D0EDB7FEB7319623E10D
:1003B00032E0ADB7BEB712963C932E931197898168
:1003C000828313829ED70F900F900F900F9080E939
:1003D00088DFFFCF90912B012DB73EB728503040DA
:1003E0000FB6F8943EBF0FBE2DBFEDB7FEB73196E6
:1003F0002DEB31E0ADB7BEB712963C932E9311971B
:100400008283138264831582968317827AD72DB7ED
:100410003EB7285F3F4F0FB6F8943EBF0FBE2DBFCB
:1004200080E95FCF1F93DF93CF9300D00F92CDB7BA
:10043000DEB780912B018B3009F087C086EA91E00E
:100440007FD730D1182F8823E9F0813019F48CE759
:1004500091E002C085E691E073D700D000D0EDB7FF
:10046000FEB731962BE431E0ADB7BEB712963C93A0
:100470002E9311971283138244D70F900F900F90F1
:100480000F904AC081E082D3882341F000D000D091
:10049000EDB7FEB7319628E031E00EC080911C0127
:1004A00060911D0189D3882379F000D000D0EDB789
:1004B000FEB7319621EB30E0ADB7BEB712963C9354
:1004C0002E9311978283D7CF20911E0182E28093D1
:1004D000230181E08093240180E091E09093260144
:1004E00080932501209327011092280183E090E05A
:1004F00090932A0180932901DE011196E0E0F1E05A
:1005000083E001900D928150E1F71092A700CE0197
:100510000196B7D5882329F080E9E3DE10922B01FC
:1005200014C082E080936E009CE797BD84BD85BDBA
:100530003E9A81EF8093900089E08093910088E952
:1005400090E0FED68CE080932B010F900F900F90DF
:10055000CF91DF911F910895C9DE8EE792E0F0D62A
:1005600080E1BFDE78945EDFA2D6FDCF1F920F92AE
:100570000FB60F920BB60F9211241F932F933F9338
:100580004F935F936F937F938F939F93AF93BF939B
:10059000EF93FF931091A700177081E08093A7005D
:1005A0008091A9008F7B8093A9008091A60080FF95
:1005B0002BC08091AF004091AF008091A60085FDD7
:1005C00005C08091A6008E778093A600842F99277E
:1005D00087FD909520E830E082279327909399003B
:1005E00080939800413144F4493044F4453044F458
:1005F000433044F480E007C080EF05C080EB03C0C7
:1006000080E301C080E16DDE8091A9008064809369
:10061000A9001093A700FF91EF91BF91AF919F9117
:100620008F917F916F915F914F913F912F911F918A
:100630000F900BBE0F900FBE0F901F901895FC01EE
:100640008181843049F48581813031F48681813023
:1006500019F48781882311F082E0089580E00895DD
:10066000FC018181843049F48581813031F48681B7
:10067000823019F48781882311F082E0089580E0A8
:100680000895FC018181853029F483818370813054
:1006900019F404C0843021F082E0089580E00895C8
:1006A00081E00895AF92BF92CF92DF92EF92FF92D6
:1006B0000F931F93DF93CF93CDB7DEB7C450D240D3
:1006C0000FB6F894DEBF0FBECDBFAE014B5F5F4FDC
:1006D0005A83498323E0E22EF12CEC0EFD1E81E0CB
:1006E000B70120E032E009D4853009F45CC08630DF
:1006F00061F0882361F400E010E0CC24DD24570190
:100700007E010894E11CF11C07C083E04FC081E02A
:100710004DC09C01032F182FC114D10441F0C50115
:10072000B70141E453E040D4882351F41CC0C50113
:10073000B7014FE153E038D48823B9F5C980DA8096
:10074000C501B70140E353E02FD4882349F0C50128
:10075000B7014FE153E028D4882339F5C980DA8006
:1007600009811A8135C0E981FA81828187FF30C011
:10077000902F812F309769F2D80112968C911297A1
:1007800080931C0113968C9180931D0122812093EC
:100790001E010481158181E061E040E194E0E92ED1
:1007A00022D280E003C082E001C084E0CC5FDD4F54
:1007B0000FB6F894DEBF0FBECDBFCF91DF911F9172
:1007C0000F91FF90EF90DF90CF90BF90AF90089582
:1007D000902F812F9ECF80919E0090E0817090702D
:1007E0002091A0002D7F2093A00020919E002260E8
:1007F00020939E0020919E0021FDFCCF20919E0021
:10080000216020939E002091A00030E02072307083
:100810004091A0004F7D4093A00040919F004F7DEC
:1008200040939F004AE050919F0055FF0BC04091BC
:100830009F004F7D40939F0040919F004D7F4093CC
:100840009F0008C0EFECF7E03197F1F700C000001F
:10085000415049F72115310529F02091A00020626F
:100860002093A000009729F480919E008E7F8093B2
:100870009E008091A00082608093A0000895409126
:100880009E0050E0417050702091A00030E0207236
:1008900030709091A0009F7D9093A00090919F0058
:1008A0009F7D90939F0090919E00916090939E00F9
:1008B00026C090919F0095FF06C090919F009F7D5C
:1008C00090939F00815090912B019230D9F090919C
:1008D000A60094FF09C01092F5008091A6008F7EBB
:1008E0008093A60082E00FC09091A60091FF07C000
:1008F0008091A6008D7F8093A60083E004C08823AA
:10090000C1F601C081E04115510529F490919E0086
:100910009E7F90939E002115310529F09091A000B3
:1009200090629093A0000895EF920F931F93DF932E
:10093000CF93CDB7DEB728970FB6F894DEBF0FBEC2
:10094000CDBF80912B01863009F499C0873070F4B7
:100950008330C9F1843020F4813009F00BC113C019
:100960008430C9F1853009F005C160C0883009F4D0
:10097000A0C0883008F48FC0893009F4B9C08A302B
:1009800009F0F8C0DEC0009120011091210101158D
:10099000110509F4EFC081E072DF682F882331F080
:1009A00080911F0180932B0181E0E0C00150104035
:1009B00010932101009320010115110509F0DAC0FF
:1009C00080911F01C3C088EE93E090932101809332
:1009D000200184E0BBC080912001909121019C0105
:1009E000215030403093210120932001009739F0AD
:1009F0008FEC97E00197F1F700C00000BBC077983B
:100A00008091D80080618093D8008091DD008B7F39
:100A10008093DD008091D70080618093D700809122
:100A2000DD0082608093DD0085E090C080919F00B2
:100A300080FFA0C080919F008E7F80939F00809157
:100A40009F008D7F80939F008091DF008D7F80933A
:100A5000DF008091DE0082608093DE0080919E0046
:100A6000816080939E0026D181E080932B0184E6F3
:100A700090E0909321018093200186E05FC0ABDE7F
:100A800081E080932B0188EC90E09093210180938A
:100A9000200187E053C080E060E040E020E000E417
:100AA00010E0EE24A0D08091AC0087FF5BC088E00E
:100AB0004DC0A3E2B1E0E3E1F1E088E001900D92E6
:100AC0008150E1F7CE010196DCD2682F882309F02E
:100AD0004CC0888580931B017EDE81E080932B01D2
:100AE00088EC90E0909321018093200189E026C05A
:100AF00000911B0180E060E040E020E010E0EE2487
:100B000072D08091AC0087FF2DC0A3E2B1E0EBE092
:100B1000F1E088E001900D928150E1F780E090E0F3
:100B2000B0D2682F882309F581E080932B0184E6F9
:100B300090E090932101809320018AE080931F012F
:100B400019C081E08093A10024DC8BE080932B010D
:100B500011C040DC8091DD0081608093DD0014DCF9
:100B6000D5D008C060E084E001C083E090912B0103
:100B7000923079F728960FB6F894DEBF0FBECDBF3E
:100B8000CF91DF911F910F91EF9008951092230163
:100B900099E09093240180932501109226011092F0
:100BA00028011092270110922A0110922901109217
:100BB000A70080E090E065C2E3E2F1E091E090936D
:100BC00023019BE09093240160932501138280937D
:100BD0002701158210922A01109229011092A70074
:100BE00080E090E04EC2EF920F931F935E2D6295CE
:100BF000660F660F607C642B2F70622B982F5260FB
:100C00004DC09093A7009817B1F428E030E040E081
:100C100003C04F5F220F331F2017310710F44530F8
:100C2000C1F7242F2295207F252BA62F40E070E0CE
:100C3000E1E2F0E00CC0A091AA002091AB00F0919D
:100C4000AD00E091A9007091A5004091AE003091F7
:100C5000A90030623093A90021FF1FC03091A90084
:100C60003E7F3093A9003091AB0032703093AB00DF
:100C70003091A90031603093A900A093AA0020937D
:100C8000AB00F093AD00E093A9007093A5004093F2
:100C9000AE002091AC0027FF08C09F5F973008F49A
:100CA000B0CF8093A70081E001C080E01F910F9139
:100CB000EF9008951092F80080E08093A7001092C2
:100CC000AE001092A6001092AB009091A9009E7FFA
:100CD0009093A9008F5F873081F708956ED075D00B
:100CE000E0EEF0E0808181608083E8EDF0E08081DB
:100CF0008F77808319BCA7EDB0E08C918E7F8C93A9
:100D000080818F7E808310922201089556D05DD01D
:100D10008091D800982F9F779093D8008068809317
:100D2000D8008091D8008F7D8093D8008091D70023
:100D30008F778093D7008CE089BD89B5826089BDAB
:100D400009B400FEFDCF82E080932B0180E4809304
:100D50001B018091D80080648093D8008091DD00D1
:100D600081608093DD008091DD0084608093DD00F0
:100D70008091D7008F7E8093D7006F9A779A809169
:100D8000DE0081608093DE008091DE0084608093CD
:100D9000DE008091E0008E7F8093E0008091D8009B
:100DA00080618093D8000895E7EDF0E08081816054
:100DB000808381E080932201A9CFE8EDF0E080817B
:100DC0008C7F80831092A00008951092DA00109218
:100DD0009F0008951F920F920FB60F920BB60F92BD
:100DE00011242F933F934F935F936F937F938F9330
:100DF0009F93AF93BF93EF93FF9380919F0085FFE5
:100E00000AC08091A00085FF06C080919F008F7D61
:100E100080939F000CD180919F0081FF15C080912D
:100E2000A00081FF11C080919F008D7F80939F0063
:100E300080919F008E7F80939F008091A0008D7F86
:100E40008093A000A1DA62DF8091DF0081FF15C0EE
:100E50008091DE0081FF11C08091DF008D7F809343
:100E6000DF0077988091DD0081608093DD0080E075
:100E700092DA8ADA82E080932B018091DF0080FF92
:100E800017C08091DE0080FF13C08091DF008E7F4D
:100E90008093DF008091DE008E7F8093DE006FDA2A
:100EA0008091A00082608093A00083E080932B015A
:100EB0008091DF0082FF0EC08091DE0082FF0AC0B9
:100EC0008091DF008B7F8093DF0082E060E082DA38
:100ED0005BDA1CDFFF91EF91BF91AF919F918F91F2
:100EE0007F916F915F914F913F912F910F900BBE2A
:100EF0000F900FBE0F901F901895CF92DF92EF9238
:100F0000FF920F931F93DF93CF93CDB7DEB729974F
:100F10000FB6F894DEBF0FBECDBF6B018A01790119
:100F200090E89093230196E09093240190E001973C
:100F300092609093260180932501109228011092CF
:100F4000270189E090E090932A0180932901109273
:100F5000A700CE01019695D08823B9F48B819C819E
:100F6000F60191838083E816F90670F090932A01C8
:100F700080932901C80185D0882339F4F801918133
:100F8000923019F086E001C085E029960FB6F894FA
:100F9000DEBF0FBECDBFCF91DF911F910F91FF90AC
:100FA000EF90DF90CF900895AF92BF92CF92DF92F3
:100FB000EF92FF920F931F93CF93DF938C01EB017E
:100FC0006A0123C0E881F9815F01208130E0C70117
:100FD0002E153F0508F4C901E80FF91FF983E883CE
:100FE000F80120813181281B390B318320838881CE
:100FF0009981F6010995823041F0813069F4A88227
:10100000B982F801F182E08207C0F801E080F18046
:10101000E114F104B9F682E0DF91CF911F910F91B5
:10102000FF90EF90DF90CF90BF90AF90089508951C
:101030001F93CF93DF93182FC8EED3E007C081E052
:101040001EDC8823D1F42097B9F02197112329F4CD
:101050008091A60083FFF3CF0DC0113029F4809159
:10106000A60080FFECCF06C0123049F78091A600A1
:1010700082FFE5CF80E001C084E0DF91CF911F9136
:101080000895EF92FF920F931F93CF93DF938C01FC
:10109000E0909E00FF2481E0E822FF24C091290116
:1010A000D0912A0180919E00816080939E0081E012
:1010B000E6DB882309F0E2C08091AA008F7C809350
:1010C000AA001092F5008091A6008F7E8093A60062
:1010D0008091A9008F7B8093A90080912301809348
:1010E000AF00809124018093AF0090912501809101
:1010F00026019093AF008093AF00909127018091DB
:1011000028019093AF008093AF00909129018091C6
:101110002A019093AF008093AF008091A60087775B
:101120008093A60080E084DF882309F0A7C0809127
:10113000A90080648093A90081E0A1DB882309F0E5
:101140009DC08091230187FF4FC08091AA008F7CB2
:1011500080618093AA000115110561F52DC0809171
:10116000A9008F7B8093A90081E062DF882309F0CA
:1011700085C08091F6009091F700009749F4C0E097
:10118000D0E006C08091AF00F80181938F012197D4
:101190008091F6009091F700009711F0209791F759
:1011A0008091A90080648093A9008091A6008E7729
:1011B0008093A600209799F68091AA008F7C806288
:1011C0008093AA008091A9008F7B8093A90082E080
:1011D0002FDF882309F052C08091A6008B7780937F
:1011E000A60082E025DF4AC00115110599F1809122
:1011F000AA008F7C80628093AA008091A9008F7BD7
:101200008093A9001CC082E013DF8823B9F5F801A0
:1012100006C081918F018093AF00219759F08F0113
:101220002091F6003091F70080911B0190E0281783
:10123000390778F38091A6008B778093A6002097DA
:1012400011F782E0F5DE8823C9F48091A90080645B
:101250008093A9008091AA008F7C80618093AA006E
:101260008091A9008F7B8093A90081E0E1DE882333
:1012700029F49091A6009E779093A6009091A900E2
:1012800090649093A900E114F10429F490919E00D8
:101290009E7F90939E0091E09093A8001092A800EA
:1012A000DF91CF911F910F91FF90EF9008951F93C1
:1012B000CF93DF93C7EAD0E018811770188234DB30
:1012C0001883DF91CF911F9108959091C80095FFE9
:1012D000FCCF8093CE0080E090E008958091C8001C
:1012E00087FF08C08091C80087FF07C02091CE000B
:1012F00030E005C02EEF3FEF02C02FEF3FEFC901F6
:101300000895DF93CF93CDB7DEB7FE013596619197
:10131000719180913C0190913D01DC0113962C91DB
:101320001397286013962C93AF0142D0E0913C01B3
:10133000F0913D012381277F2383CF91DF91089591
:10134000EF92FF920F931F93CF93DF938C01E09165
:101350003C01F0913D01838181FF20C0C0E0D0E0DD
:101360000CC0DB011896ED91FC9119970995009737
:1013700011F0CFEFDFEF0F5F1F4FF8018491609105
:101380003C0170913D01882361F7DB011896ED91D6
:10139000FC9119978AE00995009711F0CFEFDFEFE4
:1013A000CE01DF91CF911F910F91FF90EF900895A3
:1013B0002F923F924F925F926F927F928F929F9265
:1013C000AF92BF92CF92DF92EF92FF920F931F9353
:1013D000DF93CF93CDB7DEB72C970FB6F894DEBF6F
:1013E0000FBECDBF6C011B018A01FC011782168262
:1013F000838181FFC4C12E010894411C511CF60158
:101400009381F10193FD859193FF81911F018823C1
:1014100009F4B1C1853239F493FD859193FF81912F
:101420001F01853221F490E0B601DBD1E8CFEE2434
:10143000FF2420E02032B0F48B3269F08C3228F4A3
:10144000803251F0833271F40BC08D3239F0803329
:1014500049F421602CC02260246029C0286027C084
:10146000206125C027FD2CC0382F30533A3098F426
:1014700026FF08C08E2D880FE82EEE0CEE0CE80E2D
:10148000E30E15C08F2D880FF82EFF0CFF0CF80E01
:10149000F30E20620CC08E3221F426FD6CC1206454
:1014A00006C08C3611F4206802C0883649F4F10178
:1014B00093FD859193FF81911F01882309F0BACF95
:1014C000982F9554933018F09052933028F40C5F75
:1014D0001F4FFFE3F9830DC0833631F0833771F07E
:1014E000833509F05CC021C0F801808189830E5FDB
:1014F0001F4F420171E0A72EB12C15C062E0662E8D
:10150000712C600E711EF8018080918026FF03C04F
:101510006E2D70E002C06FEF7FEFC4012C8756D1B3
:101520005C0183012C852F7716C052E0652E712C4B
:10153000600E711EF8018080918026FF03C06E2D21
:1015400070E002C06FEF7FEFC4012C8734D15C01E3
:101550002C852068830123FD1EC007C080E290E037
:10156000B6012C873ED1FA942C858F2D90E0A816D9
:10157000B906A0F310C0F40127FD859127FF8191E2
:101580004F0190E0B6012C872CD12C85F110FA94F4
:101590000894A108B108A114B10469F7E9C0843620
:1015A00011F0893641F527FF08C0F801608171818B
:1015B000828193810C5F1F4F09C0F80160817181A6
:1015C000882777FD8095982F0E5F1F4F4FE6B42E2A
:1015D000B22297FF09C090958095709561957F4FD5
:1015E0008F4F9F4FF0E8BF2AA2012AE030E025D1BB
:1015F000782E741844C0853731F43FEEB32EB222F2
:101600002AE030E025C099EFB92EB2228F36C1F022
:10161000803720F4883509F0AEC00DC0803721F046
:10162000883709F0A8C002C020E1B22AB4FE0BC07E
:1016300084E0B82A08C0B4FE09C0E6E0BE2A06C0AD
:1016400028E030E005C020E130E002C020E132E0D7
:10165000B7FE08C0F80160817181828193810C5FBF
:101660001F4F07C0F8016081718180E090E00E5F3C
:101670001F4FA201E2D0782E7418FFE7BF22B6FEFA
:101680000BC02EEFB2227E1438F4B4FE07C0B2FCB9
:1016900005C08FEEB82202C0A72C01C0AE2C8B2D46
:1016A00090E0B4FE0DC0FE01E70DF11D2081203356
:1016B00019F4E9EEBE2209C0A394B2FE06C004C02C
:1016C00086789070009709F0A3948B2C9924B3FC32
:1016D00013C0B0FE0EC0AF1428F4E72CEF0CEA18CC
:1016E000AF2C07C0E72C05C080E290E0B60179D0AE
:1016F000A394AF14C8F304C0AF1410F4FA1801C0D7
:10170000FF2484FE0EC080E390E0B6016AD082FE22
:101710001DC081FE03C088E590E010C088E790E01E
:101720000DC0C40186789070009781F081FC02C0E2
:1017300080E201C08BE2B7FC8DE290E0B60151D0AF
:1017400005C080E390E0B6014CD0EA947E14C8F363
:101750007A94F201E70DF11D808190E0B60141D04D
:101760007720B1F705C080E290E0B6013AD0FA9454
:10177000FF20C9F744CEF6012681378102C02FEF42
:101780003FEFC9012C960FB6F894DEBF0FBECDBF58
:10179000CF91DF911F910F91FF90EF90DF90CF904D
:1017A000BF90AF909F908F907F906F905F904F9081
:1017B0003F902F900895FC010590615070400110FA
:1017C000D8F7809590958E0F9F1F0895FC0161506A
:1017D000704001900110D8F7809590958E0F9F1F53
:1017E00008950F931F93CF93DF938C01EB018B81AF
:1017F00081FF1BC082FF0DC02E813F818C819D81A6
:101800002817390764F4E881F9810193F983E883A3
:1018100006C0E885F985802F0995009731F48E81FF
:101820009F8101969F838E8302C00FEF1FEFC80137
:10183000DF91CF911F910F910895FA01AA272830C7
:1018400051F1203181F1E8946F936E7F6E5F7F4F8D
:101850008F4F9F4FAF4FB1E03ED0B4E03CD0670F09
:10186000781F891F9A1FA11D680F791F8A1F911D5C
:10187000A11D6A0F711D811D911DA11D20D009F4AC
:1018800068943F912AE0269F11243019305D3193EE
:10189000DEF6CF010895462F4770405D4193B3E0D7
:1018A0000FD0C9F7F6CF462F4F70405D4A3318F07E
:1018B000495D31FD4052419302D0A9F7EACFB4E02F
:1018C000A6959795879577956795BA95C9F70097E7
:1018D0006105710508959B01AC010A2E0694579588
:1018E000479537952795BA95C9F7620F731F841FDF
:0A18F000951FA01D0895F894FFCF86
:1018FA0080BB008006000100001200000501000004
:0C190A0000000080060001000008004002
:00000001FF
